:020000040000FA
:02000000602876
:08000800A800030E8301A9000A
:100010000408DB008C1A1B280B118B100B108C139F
:100020000C130C118C100C105B088400290E83003B
:10003000A80E280E09008C121A08BC0098185B281C
:1000400018195B285C0803192828BC1F1B28DC0131
:10005000310830020319312831083002031C3128DD
:100060003328B101B001B00A3008A03E84003C083A
:10007000831603138000831203133C08F83C031912
:100080000A283C08FB3C03190A283C08FA3C0319DF
:100090000A283C08FC3C03190A28B0030A285E30F1
:1000A0003002031D0A28B101B001FF30DC001B281B
:0E00B000B001B1010A28181218160A280C28EF
:1000C0000030850186018A0107309F008316B73012
:1000D0008100003085000230860009309900181236
:1000E0008312981748308B00831621308C008312BE
:1000F00010308C008F018E01343090008316031372
:10010000FF30920083120313AD01B001B1018612DA
:10011000061200308500C830D72010308500C83066
:10012000D72000308500C830D72010308500181245
:1001300018168B173108300203199A28300831023B
:10014000031CA528B001B1019A28B10A3108A03ECC
:10015000840083160313000883120313A500FA30EA
:100160002502031DB828FF30AD00051286169A2817
:10017000FB302502031DC128FF30AD000512861695
:100180009A28FC302502031DC828AD0105168612E9
:10019000F8302502031D9A28FF302D02031D9A28EE
:1001A00006160430D72006120430D7209A28A10062
:1001B000FA30A20000000000000000000000000073
:1001C000000000000000000000000000000000002F
:1001D000000000000000A20BDA28A10BD828003490
:02400E00223F4F
:00000001FF
